:020000040000FA
:040000008A010C283D
:08000800A0000308A10021087B
:100010008300A00E200E0900831603133E308500D6
:10002000003086000130870081138116011681158A
:10003000011181100110831203138B138B120B1209
:100040008B11901190141012901210151010A12005
:10005000CB202030D7204630D7203530D720433032
:10006000D7204130D7205530D720FA307F20FA30C2
:100070007F20FA307F20FA307F20F8207630D7209A
:100080003130D7202E30D7203030D720FA307F20A3
:10009000FA307F20FA307F20FA307F208B13101047
:1000A0008F018E01101405148A2005101010AA016A
:1000B0000F08AB000E08AC00E330AC07031C662849
:1000C0000130AB07031C66280130AA070000A130ED
:1000D000AB07031C6D280130AA0700001530AA07E2
:1000E00013213C214E282330A2000000A20B7528CA
:1000F00008001130A3007320A30B7B280800A60082
:100100007920A60B80280800F230A7000000A70B7A
:10011000862808000030A8008420A80B8C281B30FB
:10012000A90000000000A90B9128000000000000B9
:100130000000000000000800061600000612000083
:1001400008000F30A6007F20861206120613283002
:100150007F20061206137320023086009C20732035
:10016000023086009C207320083086009C2073207B
:10017000003086009C2073200E3086009C20732067
:10018000003086009C207320063086009C2073205F
:1001900006170612080086120613061200308600A3
:1001A0009C20013086009C2002307F200800A400A3
:1001B000A500861206170612A40CA40CA40CA40C0D
:1001C000A4132417A41224122408860010388600D1
:1001D000EF3986002508A400A4132417A4122412C2
:1001E0002408860010388600EF3986007320080046
:1001F0000A308600061206160000061200000000F3
:1002000000000000000000000830860006120616FC
:1002100000000612000000000000000000000000C6
:100220002030D720080003101830B100B001AF0112
:10023000AE01AD01AC0DAB0DAA0DB00DAF0DAE0D05
:10024000AD0DB10B242900342D30840031212E3026
:10025000840031212F30840031213030840031215D
:100260001A2903300007B200B219800030300007AD
:10027000B200B21B80000034F8202D0850212E0857
:100280004E212E0850212F084E212F0850213008D2
:100290004E212E30D720300850210800B200320EF7
:0802A0000F39303ED7200800A1
:02400E003A3D39
:00000001FF
